 ovg_unit_test

 Timestamp is 4be8d11e (Tue May 11 12:38:06 2010)

 Preferred load address is 00010000

 Start         Length     Name                   Class
 0001:00000000 00000004H .CRT$XCA                CODE
 0001:00000004 00000004H .CRT$XCZ                CODE
 0001:00000008 00000004H .CRT$XIA                CODE
 0001:0000000c 00000004H .CRT$XIZ                CODE
 0001:00000010 00000004H .CRT$XPA                CODE
 0001:00000014 00000004H .CRT$XPZ                CODE
 0001:00000018 00000004H .CRT$XTA                CODE
 0001:0000001c 00000004H .CRT$XTZ                CODE
 0001:00000020 0000057cH .rdata                  CODE
 0001:0000059c 0000002aH .rdata$debug            CODE
 0001:000005c8 000018ecH .text                   CODE
 0001:00001eb4 00000014H .xdata                  CODE
 0001:00001ec8 0000003cH .idata$2                CODE
 0001:00001f04 00000014H .idata$3                CODE
 0001:00001f18 00000148H .idata$4                CODE
 0001:00002060 00000138H .idata$6                CODE
 0001:00002198 00000000H .edata                  CODE
 0002:00000000 00000148H .idata$5                DATA
 0002:00000148 00000838H .data                   DATA
 0002:00000980 00000020H .bss                    DATA
 0003:00000000 00000090H .pdata                  DATA

  Address         Publics by Value              Rva+Base       Lib:Object

 0000:00000000       ___safe_se_handler_table   00000000     <absolute>
 0000:00000000       ___safe_se_handler_count   00000000     <absolute>
 0001:00000000       __xc_a                     00011000     corelib0:crt0init.obj
 0001:00000004       __xc_z                     00011004     corelib0:crt0init.obj
 0001:00000008       __xi_a                     00011008     corelib0:crt0init.obj
 0001:0000000c       __xi_z                     0001100c     corelib0:crt0init.obj
 0001:00000010       __xp_a                     00011010     corelib0:crt0init.obj
 0001:00000014       __xp_z                     00011014     corelib0:crt0init.obj
 0001:00000018       __xt_a                     00011018     corelib0:crt0init.obj
 0001:0000001c       __xt_z                     0001101c     corelib0:crt0init.obj
 0001:0000003c       ??_C@_0BA@ECMACICF@EGL_BAD_SURFACE?$AA@ 0001103c     ovgtest.obj
 0001:0000004c       ??_C@_0BC@OMABNJPB@EGL_BAD_PARAMETER?$AA@ 0001104c     ovgtest.obj
 0001:00000060       ??_C@_0BG@JCAPPMPM@EGL_BAD_NATIVE_WINDOW?$AA@ 00011060     ovgtest.obj
 0001:00000078       ??_C@_0BG@IANPFEBH@EGL_BAD_NATIVE_PIXMAP?$AA@ 00011078     ovgtest.obj
 0001:00000090       ??_C@_0O@GCFMIHO@EGL_BAD_MATCH?$AA@ 00011090     ovgtest.obj
 0001:000000a0       ??_C@_0BA@KHKFAGME@EGL_BAD_DISPLAY?$AA@ 000110a0     ovgtest.obj
 0001:000000b0       ??_C@_0BI@KBFIGPCO@EGL_BAD_CURRENT_SURFACE?$AA@ 000110b0     ovgtest.obj
 0001:000000c8       ??_C@_0BA@FPCJCEFK@EGL_BAD_CONTEXT?$AA@ 000110c8     ovgtest.obj
 0001:000000d8       ??_C@_0P@HOPKKPDK@EGL_BAD_CONFIG?$AA@ 000110d8     ovgtest.obj
 0001:000000e8       ??_C@_0BC@NLAJAPHP@EGL_BAD_ATTRIBUTE?$AA@ 000110e8     ovgtest.obj
 0001:000000fc       ??_C@_0O@PGDEJDGL@EGL_BAD_ALLOC?$AA@ 000110fc     ovgtest.obj
 0001:0000010c       ??_C@_0P@ELJNOEME@EGL_BAD_ACCESS?$AA@ 0001110c     ovgtest.obj
 0001:0000011c       ??_C@_0BE@JIJLFFAN@EGL_NOT_INITIALIZED?$AA@ 0001111c     ovgtest.obj
 0001:00000130       ??_C@_0M@JFIJMCIK@EGL_SUCCESS?$AA@ 00011130     ovgtest.obj
 0001:0000013c       ??_C@_03OKPHJIKM@bio?$AA@  0001113c     ovgtest.obj
 0001:00000178       ??_C@_0CN@GENKFHAM@?$CK?$CK?$CK?$CK?5VG_UNSUPPORTED_IMAGE_FORMAT@ 00011178     ovgtest.obj
 0001:000001a8       ??_C@_0CM@OIACNCNK@?$CK?$CK?$CK?$CK?5VG_UNSUPPORTED_PATH_FORMAT_@ 000111a8     ovgtest.obj
 0001:000001d4       ??_C@_0CB@IDIOOIMH@?$CK?$CK?$CK?$CK?5VG_IMAGE_IN_USE_ERROR?5?$CK?$CK?$CK?$CK?6@ 000111d4     ovgtest.obj
 0001:000001f8       ??_C@_0BP@DJDJDCNG@?$CK?$CK?$CK?$CK?5VG_NO_CONTEXT_ERROR?5?$CK?$CK?$CK?$CK?6?$AA@ 000111f8     ovgtest.obj
 0001:00000218       ??_C@_0CE@MEMLBLMJ@?$CK?$CK?$CK?$CK?5VG_PATH_CAPABILITY_ERROR?5?$CK?$CK@ 00011218     ovgtest.obj
 0001:0000023c       ??_C@_0BP@NGGBHMPE@?$CK?$CK?$CK?$CK?5VG_BAD_HANDLE_ERROR?5?$CK?$CK?$CK?$CK?6?$AA@ 0001123c     ovgtest.obj
 0001:0000025c       ??_C@_0CF@LFHIBPNG@?$CK?$CK?$CK?$CK?5VG_ILLEGAL_ARGUMENT_ERROR?5?$CK@ 0001125c     ovgtest.obj
 0001:00000284       ??_C@_0CC@CDMNEDJI@?$CK?$CK?$CK?$CK?5VG_OUT_OF_MEMORY_ERROR?5?$CK?$CK?$CK?$CK@ 00011284     ovgtest.obj
 0001:000002a8       ??_C@_0CF@GLNKALBC@?8?$CFs?8?5returned?5egl?5error?5?8?$CFs?8?5?$CI0x@ 000112a8     ovgtest.obj
 0001:000002d0       ??_C@_0P@PNPBPNLI@eglMakeCurrent?$AA@ 000112d0     ovgtest.obj
 0001:000002e0       ??_C@_0BB@KEKMNHDF@eglCreateContext?$AA@ 000112e0     ovgtest.obj
 0001:000002f4       ??_C@_0BH@MDMCFBDG@eglCreateWindowSurface?$AA@ 000112f4     ovgtest.obj
 0001:0000030c       ??_C@_0BA@GKADIFMO@eglChooseConfig?$AA@ 0001130c     ovgtest.obj
 0001:0000031c       ??_C@_0O@OMNEJBKO@eglGetConfigs?$AA@ 0001131c     ovgtest.obj
 0001:0000032c       ??_C@_0O@EEJFKEKH@eglInitialize?$AA@ 0001132c     ovgtest.obj
 0001:0000033c       ??_C@_0O@BMJFLKOA@eglGetDisplay?$AA@ 0001133c     ovgtest.obj
 0001:00000350       ??_C@_1EI@KHNCANBJ@?$AAF?$AAa?$AAi?$AAl?$AAe?$AAd?$AA?5?$AAt?$AAo?$AA?5?$AAc?$AAr?$AAe?$AAa?$AAt?$AAe?$AA?5?$AAt?$AAh?$AAe?$AA?5?$AAd?$AAe?$AAv?$AAi?$AAc?$AAe?$AA?5?$AAc?$AAo?$AAn?$AAt@ 00011350     wince_unittests.obj
 0001:00000398       ??_C@_1BO@KHIAJBLA@?$AAI?$AAn?$AAi?$AAt?$AAi?$AAa?$AAl?$AAi?$AAz?$AAa?$AAt?$AAi?$AAo?$AAn?$AA?$AA@ 00011398     wince_unittests.obj
 0001:000003b8       ??_C@_1EI@HEMGLDEE@?$AAF?$AAa?$AAi?$AAl?$AAe?$AAd?$AA?5?$AAt?$AAo?$AA?5?$AAr?$AAe?$AAg?$AAi?$AAs?$AAt?$AAe?$AAr?$AA?5?$AAt?$AAh?$AAe?$AA?5?$AAw?$AAi?$AAn?$AAd?$AAo?$AAw?$AA?5?$AAc?$AAl@ 000113b8     wince_unittests.obj
 0001:00000400       ??_C@_1BM@GPEKOMLI@?$AAP?$AAV?$AAR?$AAS?$AAh?$AAe?$AAl?$AAl?$AAC?$AAl?$AAa?$AAs?$AAs?$AA?$AA@ 00011400     wince_unittests.obj
 0001:0000041c       ??_C@_07CHIKDHJG@?9height?$AA@ 0001141c     wince_unittests.obj
 0001:00000424       ??_C@_06EGEBBOP@?9width?$AA@ 00011424     wince_unittests.obj
 0001:0000042c       ??_C@_05MHNCFLJI@?9posy?$AA@ 0001142c     wince_unittests.obj
 0001:00000434       ??_C@_05NOMJGKNJ@?9posx?$AA@ 00011434     wince_unittests.obj
 0001:00000440       ??_C@_1KE@BDGMONOJ@?$AAH?$AA?3?$AA?2?$AAW?$AAI?$AAN?$AAC?$AAE?$AA6?$AA0?$AA0?$AA?2?$AAP?$AAL?$AAA?$AAT?$AAF?$AAO?$AAR?$AAM?$AA?2?$AAS?$AAM?$AAD?$AAK?$AAV?$AA2?$AA1?$AA0?$AA?2?$AAS?$AAR@ 00011440     wince_unittests.obj
 0001:000004e4       ??_C@_1CI@OHCJFJPM@?$AAE?$AAR?$AAR?$AAO?$AAR?$AA?3?$AA?5?$AA?$CF?$AAs?$AA?5?$AAl?$AAi?$AAn?$AAe?$AA?5?$AA?$CF?$AAd?$AA?3?$AA?5?$AA?$AA@ 000114e4     wince_unittests.obj
 0001:0000050c       ??_C@_1CK@MPGKAOE@?$AA?$CI?$AAe?$AAr?$AAr?$AAo?$AAr?$AA?5?$AAc?$AAo?$AAd?$AAe?$AA?3?$AA?5?$AA?$CF?$AAd?$AA?$CJ?$AA?3?$AA?5?$AA?$CF?$AAs?$AA?$AA@ 0001150c     wince_unittests.obj
 0001:00000538       ??_C@_1M@DMCDIEDK@?$AAP?$AAK?$AAM?$AA1?$AA?3?$AA?$AA@ 00011538     wince_unittests.obj
 0001:00000544       ??_C@_0L@GPAGIAIC@?9disablepm?$AA@ 00011544     wince_unittests.obj
 0001:00000550       ??_C@_1M@ILHOPKA@?$AAE?$AAr?$AAr?$AAo?$AAr?$AA?$AA@ 00011550     wince_unittests.obj
 0001:0000055c       ??_C@_1DG@PCJNAHOH@?$AAF?$AAa?$AAi?$AAl?$AAe?$AAd?$AA?5?$AAt?$AAo?$AA?5?$AAg?$AAe?$AAt?$AA?5?$AAm?$AAo?$AAn?$AAi?$AAt?$AAo?$AAr?$AA?5?$AAi?$AAn?$AAf?$AAo?$AA?$AA@ 0001155c     wince_unittests.obj
 0001:00000594       ??_C@_07FBLHGNAH@app?4exe?$AA@ 00011594     wince_unittests.obj
 0001:00000710       Init_Bio                   00011710 f   ovgtest.obj
 0001:000009d8       Render_Bio                 000119d8 f   ovgtest.obj
 0001:00000ebc       Deinit_Bio                 00011ebc f   ovgtest.obj
 0001:00000f50       main                       00011f50 f   ovgtest.obj
 0001:000012b8       AppWndProc                 000122b8 f   wince_unittests.obj
 0001:00001318       WinMain                    00012318 f   wince_unittests.obj
 0001:00001854       vgSetf                     00012854 f   libOpenVG:libOpenVG.dll
 0001:00001864       vgSetPaint                 00012864 f   libOpenVG:libOpenVG.dll
 0001:00001874       vgSetParameterfv           00012874 f   libOpenVG:libOpenVG.dll
 0001:00001884       vgSetParameteri            00012884 f   libOpenVG:libOpenVG.dll
 0001:00001894       vgCreatePaint              00012894 f   libOpenVG:libOpenVG.dll
 0001:000018a4       vgAppendPathData           000128a4 f   libOpenVG:libOpenVG.dll
 0001:000018b4       vgClearPath                000128b4 f   libOpenVG:libOpenVG.dll
 0001:000018c4       vgCreatePath               000128c4 f   libOpenVG:libOpenVG.dll
 0001:000018d4       vgSeti                     000128d4 f   libOpenVG:libOpenVG.dll
 0001:000018e4       vgSetfv                    000128e4 f   libOpenVG:libOpenVG.dll
 0001:000018f4       vgDrawPath                 000128f4 f   libOpenVG:libOpenVG.dll
 0001:00001904       vgScale                    00012904 f   libOpenVG:libOpenVG.dll
 0001:00001914       vgRotate                   00012914 f   libOpenVG:libOpenVG.dll
 0001:00001924       vgTranslate                00012924 f   libOpenVG:libOpenVG.dll
 0001:00001934       vgLoadIdentity             00012934 f   libOpenVG:libOpenVG.dll
 0001:00001944       vgGetError                 00012944 f   libOpenVG:libOpenVG.dll
 0001:00001954       vgClear                    00012954 f   libOpenVG:libOpenVG.dll
 0001:00001964       vgDestroyPath              00012964 f   libOpenVG:libOpenVG.dll
 0001:00001974       vgDestroyPaint             00012974 f   libOpenVG:libOpenVG.dll
 0001:00001984       GetDC                      00012984 f   coredll:COREDLL.dll
 0001:00001994       PostQuitMessage            00012994 f   coredll:COREDLL.dll
 0001:000019a4       DefWindowProcW             000129a4 f   coredll:COREDLL.dll
 0001:000019b4       ReleasePowerRequirement    000129b4 f   coredll:COREDLL.dll
 0001:000019c4       DestroyWindow              000129c4 f   coredll:COREDLL.dll
 0001:000019d4       ReleaseDC                  000129d4 f   coredll:COREDLL.dll
 0001:000019e4       CreateWindowExW            000129e4 f   coredll:COREDLL.dll
 0001:000019f4       RegisterClassW             000129f4 f   coredll:COREDLL.dll
 0001:00001a04       GetStockObject             00012a04 f   coredll:COREDLL.dll
 0001:00001a14       NKDbgPrintfW               00012a14 f   coredll:COREDLL.dll
 0001:00001a24       FormatMessageW             00012a24 f   coredll:COREDLL.dll
 0001:00001a34       GetLastError               00012a34 f   coredll:COREDLL.dll
 0001:00001a44       SetPowerRequirement        00012a44 f   coredll:COREDLL.dll
 0001:00001a54       WideCharToMultiByte        00012a54 f   coredll:COREDLL.dll
 0001:00001a64       SetCursorPos               00012a64 f   coredll:COREDLL.dll
 0001:00001a74       GetCursorPos               00012a74 f   coredll:COREDLL.dll
 0001:00001a84       MessageBoxW                00012a84 f   coredll:COREDLL.dll
 0001:00001a94       GetMonitorInfo             00012a94 f   coredll:COREDLL.dll
 0001:00001aa4       MonitorFromPoint           00012aa4 f   coredll:COREDLL.dll
 0001:00001ab4       GetSystemMetrics           00012ab4 f   coredll:COREDLL.dll
 0001:00001b44       WinMainCRTStartup          00012b44 f   corelib0:pegwmain.obj
 0001:00001c40       exit                       00012c40 f   corelib0:cexit.obj
 0001:00001c58       _exit                      00012c58 f   corelib0:cexit.obj
 0001:00001c98       __security_init_cookie     00012c98 f   corelib0:seccinit.obj
 0001:00001cf4       __security_check_cookie    00012cf4 f   corelib0:armsecgs.obj
 0001:00001d08       __gsfailure                00012d08 f   corelib0:armsecgs.obj
 0001:00001d4c       _initterm                  00012d4c f   corelib0:crt0dat.obj
 0001:00001d80       _cinit                     00012d80 f   corelib0:crt0dat.obj
 0001:00001db4       fprintf                    00012db4 f   corelib1:COREDLL.dll
 0001:00001dc4       _getstdfilex               00012dc4 f   corelib1:COREDLL.dll
 0001:00001dd4       calloc                     00012dd4 f   corelib1:COREDLL.dll
 0001:00001de4       free                       00012de4 f   corelib1:COREDLL.dll
 0001:00001df4       atol                       00012df4 f   corelib1:COREDLL.dll
 0001:00001e04       atoi                       00012e04 f   corelib1:COREDLL.dll
 0001:00001e14       _stricmp                   00012e14 f   corelib1:COREDLL.dll
 0001:00001e24       _isctype                   00012e24 f   corelib1:COREDLL.dll
 0001:00001e34       malloc                     00012e34 f   corelib1:COREDLL.dll
 0001:00001e44       wcslen                     00012e44 f   corelib1:COREDLL.dll
 0001:00001e54       memset                     00012e54 f   corelib1:COREDLL.dll
 0001:00001e64       _XcptFilter                00012e64 f   corelib1:COREDLL.dll
 0001:00001e74       __C_specific_handler       00012e74 f   corelib1:COREDLL.dll
 0001:00001e84       __security_gen_cookie2     00012e84 f   corelib1:COREDLL.dll
 0001:00001e94       __report_gsfailure         00012e94 f   corelib1:COREDLL.dll
 0001:00001ea4       TerminateProcess           00012ea4 f   coredll:COREDLL.dll
 0001:00001ec8       __IMPORT_DESCRIPTOR_libOpenVG 00012ec8     libOpenVG:libOpenVG.dll
 0001:00001edc       __IMPORT_DESCRIPTOR_libEGL 00012edc     libEGL:libEGL.dll
 0001:00001ef0       __IMPORT_DESCRIPTOR_COREDLL 00012ef0     coredll:COREDLL.dll
 0001:00001f04       __NULL_IMPORT_DESCRIPTOR   00012f04     libOpenVG:libOpenVG.dll
 0002:00000000       __imp_ReleaseDC            00014000     coredll:COREDLL.dll
 0002:00000004       __imp___report_gsfailure   00014004     corelib1:COREDLL.dll
 0002:00000008       __imp___security_gen_cookie2 00014008     corelib1:COREDLL.dll
 0002:0000000c       __imp___C_specific_handler 0001400c     corelib1:COREDLL.dll
 0002:00000010       __imp__XcptFilter          00014010     corelib1:COREDLL.dll
 0002:00000014       __imp_memset               00014014     corelib1:COREDLL.dll
 0002:00000018       __imp_wcslen               00014018     corelib1:COREDLL.dll
 0002:0000001c       __imp_malloc               0001401c     corelib1:COREDLL.dll
 0002:00000020       __imp__isctype             00014020     corelib1:COREDLL.dll
 0002:00000024       __imp__stricmp             00014024     corelib1:COREDLL.dll
 0002:00000028       __imp_atoi                 00014028     corelib1:COREDLL.dll
 0002:0000002c       __imp_atol                 0001402c     corelib1:COREDLL.dll
 0002:00000030       __imp_free                 00014030     corelib1:COREDLL.dll
 0002:00000034       __imp___muls               00014034     corelib1:COREDLL.dll
 0002:00000038       __imp___dtos               00014038     corelib1:COREDLL.dll
 0002:0000003c       __imp___addd               0001403c     corelib1:COREDLL.dll
 0002:00000040       __imp___muld               00014040     corelib1:COREDLL.dll
 0002:00000044       __imp_sin                  00014044     corelib1:COREDLL.dll
 0002:00000048       __imp___stod               00014048     corelib1:COREDLL.dll
 0002:0000004c       __imp_cos                  0001404c     corelib1:COREDLL.dll
 0002:00000050       __imp___divs               00014050     corelib1:COREDLL.dll
 0002:00000054       __imp___itos               00014054     corelib1:COREDLL.dll
 0002:00000058       __imp_calloc               00014058     corelib1:COREDLL.dll
 0002:0000005c       __imp__getstdfilex         0001405c     corelib1:COREDLL.dll
 0002:00000060       __imp_fprintf              00014060     corelib1:COREDLL.dll
 0002:00000064       __imp_GetSystemMetrics     00014064     coredll:COREDLL.dll
 0002:00000068       __imp_MonitorFromPoint     00014068     coredll:COREDLL.dll
 0002:0000006c       __imp_GetMonitorInfo       0001406c     coredll:COREDLL.dll
 0002:00000070       __imp_MessageBoxW          00014070     coredll:COREDLL.dll
 0002:00000074       __imp_GetCursorPos         00014074     coredll:COREDLL.dll
 0002:00000078       __imp_SetCursorPos         00014078     coredll:COREDLL.dll
 0002:0000007c       __imp_WideCharToMultiByte  0001407c     coredll:COREDLL.dll
 0002:00000080       __imp_GetDC                00014080     coredll:COREDLL.dll
 0002:00000084       __imp_PostQuitMessage      00014084     coredll:COREDLL.dll
 0002:00000088       __imp_DefWindowProcW       00014088     coredll:COREDLL.dll
 0002:0000008c       __imp_ReleasePowerRequirement 0001408c     coredll:COREDLL.dll
 0002:00000090       __imp_DestroyWindow        00014090     coredll:COREDLL.dll
 0002:00000094       __imp_TerminateProcess     00014094     coredll:COREDLL.dll
 0002:00000098       __imp_CreateWindowExW      00014098     coredll:COREDLL.dll
 0002:0000009c       __imp_RegisterClassW       0001409c     coredll:COREDLL.dll
 0002:000000a0       __imp_GetStockObject       000140a0     coredll:COREDLL.dll
 0002:000000a4       __imp_NKDbgPrintfW         000140a4     coredll:COREDLL.dll
 0002:000000a8       __imp_FormatMessageW       000140a8     coredll:COREDLL.dll
 0002:000000ac       __imp_GetLastError         000140ac     coredll:COREDLL.dll
 0002:000000b0       __imp_SetPowerRequirement  000140b0     coredll:COREDLL.dll
 0002:000000b4       \177COREDLL_NULL_THUNK_DATA 000140b4     coredll:COREDLL.dll
 0002:000000b8       __imp_eglGetDisplay        000140b8     libEGL:libEGL.dll
 0002:000000bc       __imp_eglBindAPI           000140bc     libEGL:libEGL.dll
 0002:000000c0       __imp_eglInitialize        000140c0     libEGL:libEGL.dll
 0002:000000c4       __imp_eglGetConfigs        000140c4     libEGL:libEGL.dll
 0002:000000c8       __imp_eglChooseConfig      000140c8     libEGL:libEGL.dll
 0002:000000cc       __imp_eglCreateWindowSurface 000140cc     libEGL:libEGL.dll
 0002:000000d0       __imp_eglCreateContext     000140d0     libEGL:libEGL.dll
 0002:000000d4       __imp_eglMakeCurrent       000140d4     libEGL:libEGL.dll
 0002:000000d8       __imp_eglQuerySurface      000140d8     libEGL:libEGL.dll
 0002:000000dc       __imp_eglSwapInterval      000140dc     libEGL:libEGL.dll
 0002:000000e0       __imp_eglSwapBuffers       000140e0     libEGL:libEGL.dll
 0002:000000e4       __imp_eglTerminate         000140e4     libEGL:libEGL.dll
 0002:000000e8       __imp_eglDestroySurface    000140e8     libEGL:libEGL.dll
 0002:000000ec       __imp_eglDestroyContext    000140ec     libEGL:libEGL.dll
 0002:000000f0       __imp_eglGetError          000140f0     libEGL:libEGL.dll
 0002:000000f4       \177libEGL_NULL_THUNK_DATA 000140f4     libEGL:libEGL.dll
 0002:000000f8       __imp_vgDestroyPaint       000140f8     libOpenVG:libOpenVG.dll
 0002:000000fc       __imp_vgDestroyPath        000140fc     libOpenVG:libOpenVG.dll
 0002:00000100       __imp_vgClear              00014100     libOpenVG:libOpenVG.dll
 0002:00000104       __imp_vgGetError           00014104     libOpenVG:libOpenVG.dll
 0002:00000108       __imp_vgLoadIdentity       00014108     libOpenVG:libOpenVG.dll
 0002:0000010c       __imp_vgTranslate          0001410c     libOpenVG:libOpenVG.dll
 0002:00000110       __imp_vgRotate             00014110     libOpenVG:libOpenVG.dll
 0002:00000114       __imp_vgScale              00014114     libOpenVG:libOpenVG.dll
 0002:00000118       __imp_vgDrawPath           00014118     libOpenVG:libOpenVG.dll
 0002:0000011c       __imp_vgSetfv              0001411c     libOpenVG:libOpenVG.dll
 0002:00000120       __imp_vgSeti               00014120     libOpenVG:libOpenVG.dll
 0002:00000124       __imp_vgCreatePath         00014124     libOpenVG:libOpenVG.dll
 0002:00000128       __imp_vgClearPath          00014128     libOpenVG:libOpenVG.dll
 0002:0000012c       __imp_vgAppendPathData     0001412c     libOpenVG:libOpenVG.dll
 0002:00000130       __imp_vgCreatePaint        00014130     libOpenVG:libOpenVG.dll
 0002:00000134       __imp_vgSetParameteri      00014134     libOpenVG:libOpenVG.dll
 0002:00000138       __imp_vgSetParameterfv     00014138     libOpenVG:libOpenVG.dll
 0002:0000013c       __imp_vgSetPaint           0001413c     libOpenVG:libOpenVG.dll
 0002:00000140       __imp_vgSetf               00014140     libOpenVG:libOpenVG.dll
 0002:00000144       \177libOpenVG_NULL_THUNK_DATA 00014144     libOpenVG:libOpenVG.dll
 0002:00000148       SPIRAL2_SEGS               00014148     ovgtest.obj
 0002:00000180       SPIRAL2_VERTS              00014180     ovgtest.obj
 0002:00000350       BIOCHEM_SEGS               00014350     ovgtest.obj
 0002:000003a0       BIOCHEM_VERTS              000143a0     ovgtest.obj
 0002:00000968       gui32WindowWidth           00014968     wince_unittests.obj
 0002:0000096c       gui32WindowHeight          0001496c     wince_unittests.obj
 0002:00000970       gui32PosX                  00014970     wince_unittests.obj
 0002:00000974       gui32PosY                  00014974     wince_unittests.obj
 0002:00000978       __security_cookie          00014978     corelib0:seccinit.obj
 0002:0000097c       __security_cookie_complement 0001497c     corelib0:seccinit.obj
 0002:00000980       gbWindow                   00014980     wince_unittests.obj
 0002:00000984       ghWnd                      00014984     wince_unittests.obj
 0002:00000988       pfnRegisteredWndProc       00014988     wince_unittests.obj
 0002:0000098c       _exitflag                  0001498c     corelib0:cexit.obj
 0002:00000990       gui32DisplayWidth          00014990     <common>
 0002:00000994       gui32DisplayHeight         00014994     <common>
 0002:00000998       __onexitend                00014998     <common>
 0002:0000099c       __onexitbegin              0001499c     <common>

 entry point at        0001:00001b44

 Static symbols

 0001:000005c8       VG_ERROR_TEST              000115c8 f   ovgtest.obj
 0001:00000ef4       handle_egl_error           00011ef4 f   ovgtest.obj
 0001:00001acc       WinMainCRTStartupHelper    00012acc f   corelib0:pegwmain.obj
 0001:00001b78       doexit                     00012b78 f   corelib0:cexit.obj
